:100000000C9462000C948A000C948A000C948A0070
:100010000C948A000C948A000C948A000C948A0038
:100020000C948A000C948A000C948A000C948A0028
:100030000C948A000C948A000C948A000C948A0018
:100040000C94C6000C948A000C9409020C948A004B
:100050000C948A000C948A000C948A000C948A00F8
:100060000C948A000C948A000000000024002700F1
:100070002A0000000000250028002B0000000000DE
:1000800023002600290004040404040404040202DA
:100090000202020203030303030301020408102007
:1000A0004080010204081020010204081020000012
:1000B0000007000201000003040600000000000029
:1000C0000000520311241FBECFEFD4E0DEBFCDBF2E
:1000D00011E0A0E0B1E0E8E6FAE002C005900D9280
:1000E000AE30B107D9F711E0AEE0B1E001C01D922A
:1000F000A23BB107E1F710E0C4ECD0E004C02297C6
:10010000FE010E942E05C23CD107C9F70E94BF0024
:100110000C9432050C94000080910E010E947E0127
:10012000BC0190931101809310018FE991E00E942E
:1001300099048091100190911101883C910584F0FF
:100140008091000161E00E94BC0162E370E080E008
:1001500090E00E941A018091000160E00E94BC01C1
:1001600008958FE991E040E05BE460E070E00E9478
:1001700046028091000161E00E949C0108950E9466
:1001800044010E94B1000E948C00FDCF1F920F928B
:100190000FB60F9211242F933F934F935F936F935A
:1001A0007F938F939F93AF93BF93209116013091CC
:1001B0001701409118015091190170911A01DA014B
:1001C000C9010296A11DB11D672F6A5F6D3730F01E
:1001D0006D57DA01C9010396A11DB11D60931A0183
:1001E0008093160190931701A0931801B093190101
:1001F0008091120190911301A0911401B091150109
:100200000196A11DB11D8093120190931301A0933B
:100210001401B0931501BF91AF919F918F917F9180
:100220006F915F914F913F912F910F900FBE0F9063
:100230001F901895EF92FF920F931F937B018C01F3
:100240008FB7F894409116015091170160911801F1
:10025000709119018FBF2FB7F8948091160190917A
:100260001701A0911801B09119012FBF841B950BA4
:10027000A60BB70BE816F9060A071B0760F71F91D4
:100280000F91FF90EF900895789484B5826084BDBB
:1002900084B5816084BD85B5826085BD85B581608A
:1002A00085BDEEE6F0E0808181608083E1E8F0E0EA
:1002B000808182608083808181608083E0E8F0E0DB
:1002C000808181608083E1EBF0E0808184608083C5
:1002D000E0EBF0E0808181608083EAE7F0E08081FC
:1002E000846080838081826080838081816080835C
:1002F0008081806880831092C10008958F709091F2
:1003000002019295990F990F907C982B90937C0005
:1003100080917A00806480937A0080917A0086FDD3
:10032000FCCF2091780040917900942F80E030E05C
:10033000282B392BC9010895282F30E0C901865692
:100340009F4FFC0194912A573F4FF90184918823D4
:1003500091F0E82FF0E0EE0FFF1FE859FF4FA59155
:10036000B491662329F48C91909589238C930895F8
:100370008C91892B8C930895482F50E0CA018255A7
:100380009F4FFC012491CA0186569F4FFC01949116
:100390004A575F4FFA0134913323D1F1222331F1CF
:1003A000233021F4809180008F7705C0243031F410
:1003B000809180008F7D8093800018C0213019F4D7
:1003C00084B58F7704C0223021F484B58F7D84BD3D
:1003D0000DC0263021F48091B0008F7705C0273002
:1003E00029F48091B0008F7D8093B000E32FF0E07E
:1003F000EE0FFF1FEE58FF4FA591B491662329F42D
:100400008C91909589238C9308958C91892B8C9352
:1004100008951F920F920FB60F9211242F933F93BE
:100420004F935F936F937F938F939F93AF93BF93FC
:10043000EF93FF934091C600E0919B01F0919C01E6
:10044000CF01019660E870E00E94C8049C01809191
:100450009D0190919E012817390739F0E55EFE4F06
:10046000408330939C0120939B01FF91EF91BF91BA
:10047000AF919F918F917F916F915F914F913F913C
:100480002F910F900FBE0F901F9018955F926F9253
:100490007F928F929F92AF92BF92CF92DF92EF9214
:1004A000FF920F931F93CF93DF93EC013A014B011F
:1004B000413281EA580787E0680780E078070CF04E
:1004C0007FC060E472E48FE090E0A40193010E9499
:1004D000FD042150304040405040CA01B90122E0A3
:1004E00030E040E050E00E94FD0459016A01A6019D
:1004F0009501209530954095509594E0220F331F3B
:10050000441F551F9A95D1F760E072E18AE790E0A9
:100510000E94FD04CA01B9012FEF30E040E050E035
:100520000E94A904A40193010E94FD04C901815005
:100530009F4F181619061CF4522E5A9403C05524C6
:100540005394521A60E874E88EE190E0A40193019C
:100550000E94FD042150304040405040CA01B90182
:1005600022E030E040E050E00E94FD04209530950C
:100570004095509583E0220F331F441F551F8A95E5
:10058000D1F760E072E18AE790E00E94FD04CA01C1
:10059000B9012FEF30E040E050E00E94A904A4012F
:1005A00093010E94FD04C90181509F4F181619063E
:1005B0001CF4822F815002C081E0821B851500F55A
:1005C000E885F98581E090E00A8802C0880F991FCC
:1005D0000A94E2F7808360E874E88EE190E0A40179
:1005E00093010E94FD042150304040405040CA0118
:1005F000B90122E030E040E050E00E94FD0404C078
:10060000E885F98510829501EC81FD813083EE81CA
:10061000FF812083EA85FB85208141E050E0CA010B
:100620000E8402C0880F991F0A94E2F7282B2083BA
:10063000EA85FB852081CA010F8402C0880F991FBB
:100640000A94E2F7282B2083EA85FB8580810888BD
:1006500002C0440F551F0A94E2F7842B8083DF9178
:10066000CF911F910F91FF90EF90DF90CF90BF90AF
:10067000AF909F908F907F906F905F900895FC0156
:10068000A085B18521898C9190E0022E02C09595BC
:1006900087950A94E2F780FFF6CF0484F585E02D74
:1006A0006083089587E091E09093A00180939F017B
:1006B0008BE191E09093A2018093A10185EC90E001
:1006C0009093A4018093A30184EC90E09093A60101
:1006D0008093A50180EC90E09093A8018093A701FE
:1006E00081EC90E09093AA018093A90186EC90E0C0
:1006F0009093AC018093AB0184E08093AD0183E0E3
:100700008093AE0187E08093AF0185E08093B001D4
:1007100081E08093B10108950F931F93CF93DF93EE
:100720008C01EB0109C02196D801ED91FC9101905B
:10073000F081E02DC801099568816623A1F7DF915A
:10074000CF911F910F910895EF92FF920F931F93F6
:10075000CF93DF938C017B01EA010CC0D7016D912F
:100760007D01D801ED91FC910190F081E02DC8014F
:1007700009952197209791F7DF91CF911F910F91C4
:10078000FF90EF9008950F931F938C01DC01ED9182
:10079000FC910190F081E02D6DE00995D801ED917B
:1007A000FC910190F081E02DC8016AE009951F914C
:1007B0000F9108952F923F924F925F926F927F9286
:1007C0008F929F92AF92BF92CF92DF92EF92FF9261
:1007D0000F931F93DF93CF93CDB7DEB7A0970FB6DC
:1007E000F894DEBF0FBECDBF1C016A017B0141152D
:1007F00051056105710549F4DC01ED91FC91019011
:10080000F081E02D60E3099554C0882499245401B7
:10081000422E55246624772401E010E00C0F1D1FA2
:10082000080D191DC701B601A30192010E94DB0446
:10083000F80160830894811C911CA11CB11CC701A4
:10084000B601A30192010E94DB04C901DA016C0127
:100850007D01C114D104E104F104F1F681E0E82E38
:10086000F12CEC0EFD1EE80CF91C3E010894611CF5
:10087000711CD501C4010197A109B1096C01C81807
:10088000D90814C0F601EE0DFF1D60816A3010F426
:10089000605D01C0695CD101ED91FC910190F08136
:1008A000E02DC10109950894E108F1086E147F0458
:1008B00049F7A0960FB6F894DEBF0FBECDBFCF911B
:1008C000DF911F910F91FF90EF90DF90CF90BF903D
:1008D000AF909F908F907F906F905F904F903F90E0
:1008E0002F900895EF92FF920F931F93CF93DF9372
:1008F000EC017A018B0177FF0FC0E881F98101904B
:10090000F081E02D6DE2099510950095F094E0944A
:10091000E11CF11C011D111DCE01B801A7012AE047
:100920000E94DA03DF91CF911F910F91FF90EF901A
:1009300008950F931F938C01AB01662757FD6095B7
:10094000762F0E947204C8010E94C3031F910F9169
:100950000895629FD001739FF001829FE00DF11D09
:10096000649FE00DF11D929FF00D839FF00D749F29
:10097000F00D659FF00D9927729FB00DE11DF91FD5
:10098000639FB00DE11DF91FBD01CF011124089532
:1009900097FB092E07260AD077FD04D049D006D050
:1009A00000201AF4709561957F4F0895F6F79095A1
:1009B00081959F4F0895A1E21A2EAA1BBB1BFD0132
:1009C0000DC0AA1FBB1FEE1FFF1FA217B307E4072E
:1009D000F50720F0A21BB30BE40BF50B661F771F86
:1009E000881F991F1A9469F7609570958095909566
:1009F0009B01AC01BD01CF01089597FB092E05268F
:100A00000ED057FD04D0D7DF0AD0001C38F4509523
:100A10004095309521953F4F4F4F5F4F0895F6F722
:100A200090958095709561957F4F8F4F9F4F08955A
:100A3000AA1BBB1B51E107C0AA1FBB1FA617B70704
:100A400010F0A61BB70B881F991F5A95A9F7809520
:100A50009095BC01CD010895EE0FFF1F0590F49114
:080A6000E02D0994F894FFCF8A
:0E0A6800040001000000003F038C03A4030003
:00000001FF
